:10000000010A25003F0C0600800C02006600040077
:100010000606070A1704260617053704660637057D
:1000200004000606170A1B0C06002909100AC80C52
:100030002A00000C2B0060090607280A2F0C060076
:10004000320C2A00000C2B0060093F0C0600070A46
:10005000100A6E002606EE006F001706EF000E0273
:100060008F00000C4307C0004306440A2606430ADB
:100070003F0C0600BC0C2A00020C2B0060093B0C54
:1000800006001704440A17056E006606EE006F00AE
:100090003706EF000E028F00000C4307C000430636
:1000A000000866065E0A3F0C0600580C2A00020C87
:1000B0002B0060093B0C060037045F0A3705000877
:1000C0006C006D00090C2E001F0C2F00EF02660A59
:1000D000EE02640A280C2E00EE026C0A0400AC0248
:1000E0004306AD020A028C004307620A0B028D0030
:0600F0004307620A00084C
:0203FE00500CA1
:021FFE00EE0FE4
:00000001FF
